:100000001D288C008A010C0882070C340634033446
:1000100009348C008A010C08820708340434023445
:1000200001348C008A010C08820708340C34043433
:100030000634023403340134093410308B00283084
:100040008316810083128501103083168500831288
:100050008601FF3083168600831285018B108D0187
:1000600081018E018F0110119010101010183C2882
:100070008312861A3F2849288312861A4928831238
:10008000861E462802308D071014492802308D0242
:1000900010108B1C362810158312061E1011901C90
:1000A000101110195628010803198D280E108312FB
:1000B000061B0E148E10861B8E1403308E050E0840
:1000C00003196C28013A03197228033A0319782896
:1000D000013A03197D287D2803308D050D08012084
:1000E0008F007D2807308D050D0811208F007D2899
:1000F00003308D050D0809208F000F08831285003D
:10010000101C84288D0A85288D0383120108031989
:100110008B2881039528101195288312861992281F
:10012000850195280F08831285008B10901083128B
:06013000061A90143628A7
:00000001FF
